:0200000480007A
:1000000093000000130100009301000013020000A0
:100010009302000013030000930300001304000088
:100020009304000013050000930500001306000070
:100030009306000013070000930700001308000058
:10004000930800001309000093090000130A000040
:10005000930A0000130B0000930B0000130C000028
:10006000930C0000130D0000930D0000130E000010
:10007000930E0000130F0000930F0000B7E2010081
:1000800073A00230930210009392F20163CA02003F
:10009000130510009712000023A6A2F66FF05FFF71
:1000A00097020000938242047390523097510000EF
:1000B0009381413F177200001302B244137202FC95
:1000C000732540F1930510006370B500130115000E
:1000D0001311110133014100131615013302C2003F
:1000E0006F209041130101EF2322110023242100EE
:1000F0002326310023284100232A5100232C6100AC
:10010000232E710023208102232291022324A102A5
:100110002326B1022328C102232AD102232CE10283
:10012000232EF1022320010523221105232421057A
:100130002326310523284105232A5105232C610557
:10014000232E710523208107232291072324A10751
:100150002326B1072328C107232AD107232CE1072F
:10016000232EF10773252034F325103413060100E4
:10017000EF20901173101534B72200009382028093
:1001800073A0023083204100032181008321C1003C
:100190000322010183224101032381018323C10141
:1001A0000324010283244102032581028325C10225
:1001B0000326010383264103032781038327C10309
:1001C0000328010483284104032981048329C104ED
:1001D000032A0105832A4105032B8105832BC105D1
:1001E000032C0106832C4106032D8106832DC106B5
:1001F000032E0107832E4107032F8107832FC10799
:0802000013010111730020300D
:1010000000000000000000000000000000000000E0
:1010100000000000000000000000000000000000D0
:1010200000000000000000000000000000000000C0
:1010300000000000000000000000000000000000B0
:081040000000000000000000A8
:1020000013052500B305B5002320B6006780000046
:10201000130756001308800C330807031316260015
:10202000931727003305F5002320D500232CE50660
:102030002322D500B307C800B387F50083A60701A4
:1020400023AAE70023ACE7001387160023A8E700C4
:1020500003270500B3850501B385C500B717000048
:10206000B385B7009307500023AAE5FA173700009D
:10207000232CF7C4678000001375F50F93F5F50F57
:102080006306B50013050000678000009737000065
:10209000A388A7C21305100067800000130101FF89
:1020A000232481002322910023261100130405001C
:1020B0009384050083C5340003452400EFF0DFFB63
:1020C000E31A05FE9385040013050400EF00505940
:1020D00093070000635AA0009307A0001737000081
:1020E0002324F7BE930710008320C100032481003E
:1020F000832441001385070013010101678000005C
:102100001305E5FF1335150067800000130101FF7B
:1021100023248100232291001304050023261100AB
:1021200093840500EFF0DFFD9307040063140500BE
:102130009307300023A0F40093072000630AF404FF
:1021400063E88702630A0400173700000327C7B754
:102150009307400663DCE70423A004008320C1004A
:1021600003248100832441001301010167800000E2
:1021700013074000E314E4FE8320C1000324810020
:1021800023A0F400832441001301010167800000B3
:102190008320C100032481009307100023A0F400D2
:1021A0008324410013010101678000008320C100E6
:1021B000032481009307300023A0F400832441000E
:1021C0001301010167800000130101FE2322B10009
:1021D0002324C1002326D1002328E100232AF10073
:1021E000232C0101232E110113010102678000003D
:1021F000173700000347D7AC930710046304F700B8
:102200006780000083270500173700000327C7AB4E
:1022100093879700B387E7402320F500678000008D
:10222000973700009387C7AA03A607006308060034
:10223000032706002320E50003A607001306C600B7
:102240009735000083A545A81305A0006FF05FDB5C
:10225000130101FF2320210117390000130949A7A9
:1022600083270900232481000324050003A7070016
:1022700083AE470003AE870003A3070183A847018D
:1022800003A8870183A5070203A6470283A6870246
:1022900023229100232611009304050003A5C70102
:1022A00083A7C7022320E40003A70400232EA40071
:1022B0002326F4022322D401930750002324C401CF
:1022C00023286400232A1401232C04012320B402B0
:1022D0002322C4022324D40223A6F4002326F400DC
:1022E0002320E40013050400EFF09FF3832744004C
:1022F0006380070883A704008320C10003248100B2
:1023000083AF070003AF470083AE870003AEC7006B
:1023100003A3070183A8470103A8870183A5C70179
:1023200003A6070283A6470203A7870283A7C70263
:1023300023A0F40123A2E40123A4D40123A6C40111
:1023400023A8640023AA140123AC040123AEB40023
:1023500023A0C40223A2D40223A4E40223A6F402ED
:10236000032901008324410013010101678000005B
:1023700003A5840093076000930584002326F400DE
:10238000EFF0DFD8832709000325C4001306C4003B
:1023900083A707008320C100832441002320F40089
:1023A00003248100032901009305A000130101010A
:1023B0006FF01FC5173700001307C790832607006B
:1023C0009737000083C7D78F9387F7FB93B7170022
:1023D000B3E7D7002320F700930720041737000046
:1023E0002300F78E67800000930710041737000062
:1023F000A308F78C9737000023A6078C678000009E
:10240000130101EB23229113B70C00409387FCFFCB
:10241000232481142322911423202115232A5113CC
:1024200023261114232E3113232C41132328611347
:1024300023267113232481132320A113232EB111EA
:102440001309050093840500130406002324D1001A
:10245000930A50022326F1006F0040016304050631
:102460009385040013041400E700090003450400E9
:10247000E31655FF83461400930D140013870D00D7
:10248000930B00029309F0FF130AF0FF930500007D
:1024900013065005130590009387D6FD93F7F70FA9
:1024A00013041700636CF60617280000130808557C
:1024B00093972700B387070183A70700B387070116
:1024C000678007008320C1140324811483244114EE
:1024D000032901148329C113032A8113832A411379
:1024E000032B0113832BC112032C8112832C411265
:1024F000032D0112832DC111130101156780000006
:10250000938B06008346170013070400130417007B
:102510009387D6FD93F7F70FE378F6F893850400D9
:1025200013055002E700090013840D006FF01FF43B
:1025300003481700938906FD13070400930708FD5D
:10254000930608006366F50293972900B389370163
:102550001307170093991900B3890901034807006D
:10256000938909FD930708FD93060800E37EF5FCB7
:10257000E3540AF2138A09009309F0FF6FF0DFF1C8
:1025800083461700130704006FF01FF193850400C2
:1025900013055002E70009006FF05FED832781000B
:1025A000834617001307040083A907009387470099
:1025B0002324F1006FF0DFFB130500039385040073
:1025C000E70009009385040013058007E700090070
:1025D00083278100130C0001232201001387470089
:1025E00083278100930D000083A907002324E100C5
:1025F00013060C00930600001385090093850D0057
:10260000EF10001C2328A10093070000930C050085
:102610006380B723130B4101130D100013060C0048
:10262000930600001385090093850D00EF001056F6
:1026300013060C009306000093090500938D050016
:10264000EF100018832741002320AB002320A101B5
:10265000930C0500130B4B00130D1D00E390B7FD09
:10266000E3FE89FB635C4D01130AFAFF93850400C6
:1026700013850B00E7000900E3484DFF83270100A5
:102680000327C10093099000338AE700131A2A0038
:1026900093070101338A47016F00C000832C0A00B1
:1026A000130ACAFFB3B79901B307F04093F7770253
:1026B000938707033385970193850400E70009009A
:1026C0009307C100E39C47FD6FF05FDA93071000AA
:1026D00063CCB7160327810093074700638605186C
:1026E000832907002324F10013DCF941634E0C1801
:1026F000930D0C0023220100130CA0006FF05FEF7C
:10270000130C0001232201009307100063C2B710CD
:1027100083278100138747006FF09FEC8327810098
:1027200083AD0700138B470063840D18635840097D
:102730009307D002639EFB0403C50D0063080502E6
:10274000930BF0FF63C609009389F9FF638E79014B
:1027500093850400938D1D00E700090003C50D005B
:10276000130AFAFFE31005FE635C4001130AFAFF47
:102770009385040013050002E7000900E3180AFE30
:10278000232461016FF09FCE972D0000938D0D23C0
:1027900093870D00B3863D01639809006F004013D5
:1027A000938717006386D70003C70700E31A07FE65
:1027B000B387B741330AFA40634C401103C50D009B
:1027C000E30005FC930BF0FF6FF0DFF79347FAFF90
:1027D00093D7F74183461700337AFA0013070400B2
:1027E0006FF09FCB832781009385040003A507002A
:1027F000138B4700E7000900232461016FF01FC716
:102800008346170093851500130704006FF0DFC897
:1028100083278100138B7700137B8BFF93078B003B
:1028200083290B00832D4B002324F1006FF05FDC24
:10283000E3F289DF9307100023200100130D10003D
:10284000E3C447E36FF09FE383278100138B770096
:10285000137B8BFF93078B0083290B00032C4B000A
:102860002324F1006FF09FE8032781006FF05FE7FA
:10287000130C8000232201006FF01FE9130CA0004D
:10288000232201006FF05FE8938504001305D00256
:10289000E700090033373001B3078041B309304105
:1028A000B38DE740130CA000232201006FF05FD42A
:1028B000635640019307D002E398FBEC972D00008C
:1028C000938DCD0F13058002930BF0FF6FF09FE700
:1028D000130AFAFF9385040013850B00E700090033
:1028E000E30E0AEC130AFAFF9385040013850B002C
:1028F000E7000900E31E0AFC6FF05FEC83A7050008
:102900002380A70083A705009387170023A0F50065
:1029100067800000130101F81308F103137808FC25
:10292000130700042320E800930700002322F80087
:10293000130710002324E800930700002326F80063
:102940002328A800232AB800232CC800232ED8004F
:102950000F00F00F97E6FFFF9386C66A23A00601DB
:102960009307000023A2F60097E6FFFF9386866D8B
:1029700003A7060083A746003367F700E30A07FEB4
:102980001307000023A0E6009307000023A2F6002F
:102990000F00F00F032508008325480013010108EC
:1029A00067800000130101FF2324810083250204B6
:1029B0009307020023261100B387B7001386150082
:1029C0002380A7002320C2049307A0006300F50220
:1029D00093070004630CF6008320C10003248100E8
:1029E0001305000013010101678000009356F641B2
:1029F0001305020093050000EFF0DFF18320C10012
:102A000023200204032481001305000013010101A7
:102A100067800000732700B0972700009387072C7A
:102A2000631E050083A6070017260000130686F91B
:102A30009725000023A0C52A3307D74023A0E7002D
:102A4000732720B0631E050083A6470017260000E9
:102A50001306C6F79725000023A0C5283307D740E3
:102A600023A2E700678000009316150013E7160005
:102A700097E6FFFF938606599307000023A0E60020
:102A800023A2F6006F0000003716000097E7FFFF53
:102A900093874757130636A79306000023A0C70065
:102AA00023A2D7006F000000130101FF23261100AD
:102AB000EFF09FFB97E7FFFF9387C7541306D010F3
:102AC0009306000023A0C70023A2D7006F000000D8
:102AD000834705006382070213060500834716003B
:102AE00013061600E39C07FE3306A640930600007B
:102AF000930500006FF01FE213060000930600002C
:102B0000930500006FF01FE163100500678000006F
:102B1000130101FD13070500232611021305C1004F
:102B20001306B101130890006F00800013860700A0
:102B30009377F700B337F800B307F04093F77702C5
:102B40009376F70093870703B387F6002300F60018
:102B50009396C501135747009307F6FF33E7E60046
:102B600093D54500E314C5FC230E0100EFF05FF69A
:102B70008320C1021301010367800000130101FCDF
:102B800013034102130E05002322B1022324C102C4
:102B90002326D10217050000130505E19306030063
:102BA00013060E0093050000232E11002328E102D6
:102BB000232AF102232C0103232E11032326610073
:102BC000EFF01F848320C1011305000013010104ED
:102BD00067800000130101FB13038103232481029A
:102BE0002326A100232CC102232ED10213040500A9
:102BF0001386050017050000130585D09305C10055
:102C000093060300232611022322F1042320E1046A
:102C10002324010523261105232E6100EFF04FFE2A
:102C20008327C100238007000325C1008320C10240
:102C300033058540032481021301010567800000EC
:102C4000B3E7C500B367F50093F73700B306C500D7
:102C5000638407023386C50093070500637ED502AF
:102C600003C705009385150093871700A38FE7FE20
:102C7000E318B6FE67800000E37ED5FE93070500EB
:102C800003A70500938747009385450023AEE7FE21
:102C9000E3E8D7FE6780000067800000B367C500E7
:102CA00093F737003306C5006380070293F5F50FED
:102CB000930705006370C50493871700A38FB7FEC1
:102CC000E31CF6FE6780000093F5F50F139785006F
:102CD00033E7E500931707013367F700E374C5FE98
:102CE000930705009387470023AEE7FEE3ECC7FE9A
:102CF0006780000067800000130101F6974700001D
:102D00009387C77B23244109174A0000130A0A7BD3
:102D100023263109B309FA40232A910823282109DF
:102D2000930405001389050013050200938507002D
:102D300013860900232E1108232C81082322510910
:102D4000930A0200EFF0DFEF174600001306C67B80
:102D5000330646419305000033853A01EFF01FF436
:102D60009305090013850400EFF01FDA93050000B6
:102D700013050000EF00D06517290000130909F6BC
:102D8000832609001304F103137404FC9304050063
:102D900063940604832649006396060013850400A5
:102DA000EFF09FCC1309040097290000938989F262
:102DB00003A649001305090097250000938545C324
:102DC000EFF05FE13309A900E30A24FD13050400D5
:102DD000EFF01FD06FF09FFC97290000938989EFD7
:102DE00003A6090097250000938585C013050400FC
:102DF000EFF05FDE832649003309A400E38606FC7A
:102E00006FF01FFB83470500638E070093070500E3
:102E100003C7170093871700E31C07FE3385A740FD
:102E2000678000001305000067800000130605009E
:102E3000B306B600138505009307060063980500E6
:102E40006F00C001938717006388F60003C707006F
:102E5000E31A07FE3385C7406780000067800000E3
:102E600083470500938515001305150003C7F5FF7B
:102E700063880700E386E7FE3385E740678000004C
:102E8000930700006FF05FFF9307050003C705007D
:102E90009387170093851500A38FE7FEE31807FEBD
:102EA00067800000034705009306000293070500B2
:102EB0006318D70003C7170093871700E30CD7FEEA
:102EC0009306D0026300D7069306B0026300D704CE
:102ED00083C6070093050000638206041305000003
:102EE00093871700138606FD1317250083C6070076
:102EF0003305A700131515003305A600E39206FE5F
:102F0000638005023305A0406780000083C6170078
:102F10009305000093871700E39206FC1305000059
:102F20006780000083C61700930510009387170081
:102F3000E39606FA130500006FF09FFE138F05005D
:102F40001308000063DC0500B337A000B305B040F0
:102F5000338FF5403305A0401308F0FF63DA060015
:102F6000B335C0003307D040B306B7403306C04086
:102F700093080600138706009307050093050F00CA
:102F800063940624B7560080938606B56376CF0E09
:102F9000370301006378660C1303F00F6374C300FA
:102FA000130780003353E600B386660003CE0600A5
:102FB000330EEE00130700023303C741630CC70151
:102FC000B3156F00335EC501B3186600B365BE006C
:102FD000B317650013D60801B3F6C50213950801AF
:102FE0001355050113D70701B3D5C5029396060102
:102FF00033E7E600B305B502637AB700330717017C
:10300000636617016374B700330717013307B740CE
:10301000B376C7029397070193D707013357C702C7
:103020003307E50213950601B367F50063FAE7007D
:10303000B387170163E6170163F4E700B38717014D
:10304000B387E74033D5670093050000630A0800A3
:10305000B337A000B306B040B385F6403305A040B7
:10306000678000003703000113070001E36C66F27C
:10307000130780016FF01FF363160600930810001A
:10308000B3D8E8023706010063F6C8121306F00F42
:10309000637416011307800033D6E800B386C600B8
:1030A00003CE0600B3051F41330EEE0013070002E6
:1030B0003303C7416306C709B3986800B35ECF0105
:1030C000B3176500335EC50113D50801B3156F0052
:1030D000336EBE009395080193D5050113560E017A
:1030E000B3D6AE0233F7AE02B386D502131707018B
:1030F0003367C700637AD700330717016366170188
:103100006374D700330717013306D7403377A6021D
:10311000131E0E01135E0E013356A602131707018C
:103120003386C502B365C70163FAC500B3851501CF
:1031300063E6150163F4C500B3851501B385C54089
:1031400093D6080133F7D5021395080113550501ED
:1031500013D60701B3D5D502131707013367C7008C
:10316000B305B502637AB700330717016366170129
:103170006374B70033071701B305B74033F7D502BF
:103180009397070193D70701B3D5D502B305B502CD
:1031900013150701B367F50063FAB700B38717018A
:1031A00063E6170163F4B700B3871701B387B7402D
:1031B0006FF05FE93706000113070001E3EEC8EC8A
:1031C000130780016FF05FEDE362DFE8370701006E
:1031D00063FAE604930EF00F33B7DE0013173700DF
:1031E000B758008033D3E600938808B5B3886800E9
:1031F00083CE0800B38EEE0013070002330ED741D2
:10320000631CD70363E4E601636AC500B307C540E6
:10321000B305DF403335F500B385A54013850700BE
:103220006FF0DFE2B708000113070001E3EA16FBC5
:10323000130780016FF0DFFA3357D601B396C6014A
:10324000B36FD700B357DF0113D70F0133F3E70292
:10325000B315CF01B356D501B3E6B60093950F0170
:1032600093D5050193D806013316C6013315C50160
:10327000B3D7E70213130301B3681301338FF502C9
:103280001383070063FEE801B388F8011383F7FF97
:1032900063E8F80163F6E8011383E7FFB388F801F8
:1032A000B388E84133FFE8029396060193D60601FE
:1032B000B3D8E802131F0F01336FDF00B385150386
:1032C00093870800637EBF00330FFF019387F8FFE9
:1032D0006368FF016376BF009387E8FF330FFF0148
:1032E000B305BF4013130301370F01003363F3002D
:1032F0009307FFFFB378F3009356060113530301BE
:10330000B377F6003387F802B307F302B388D80225
:103310003303D302B388F80093560701B38616012E
:1033200063F4F6003303E30193D7060133836700A8
:10333000B70701009387F7FFB3F6F60093960601EF
:103340003377F7003387E60063E66500639E650028
:10335000637CE5003306C7403337C7003307F70106
:103360003303E340130706003307E5403335E50038
:10337000B3856540B385A540B397D5013357C701E1
:1033800033E5E700B3D5C5016FF05FCC93080500C6
:1033900093870500130806001385060013830800B1
:1033A00063940628B7560080938606B563F6C50E6B
:1033B000370701006378E60C1307F00F3337C700B7
:1033C000131737003355E600B386A60083C6060000
:1033D000130500023387E600B306E540630CE50001
:1033E000B397D70033D7E8003318D600B365F7009A
:1033F0003393D80093580801B3D715031316080167
:103400001356060113570301B3F61503138507007E
:10341000B305F6029396060133E7E600637EB70034
:10342000330707011385F7FF636807016376B70069
:103430001385E7FF330707013307B740B377170357
:103440001313030113530301335717039397070112
:1034500033E36700B306E60213060700637CD3007C
:10346000330368001306F7FF636603016374D30038
:103470001306E7FF131505013365C500930500002A
:103480006F00400E3705000113070001E36CA6F240
:10349000130780016FF01FF3631606001307100077
:1034A0003358C702370701006370E80C1307F00FA9
:1034B00063740701130580003357A800B386E60044
:1034C00003C70600130600023307A700B306E64051
:1034D0006316E60AB3870741930510009358080165
:1034E000131608011356060113570301B3F6170309
:1034F000B3D717039396060133E7E600330EF602BF
:1035000013850700637EC701330707011385F7FFA3
:10351000636807016376C7011385E7FF3307070177
:103520003307C741B3771703131303011353030181
:10353000335717039397070133E36700B306E60297
:1035400013060700637CD300330368001306F7FFFC
:10355000636603016374D3001306E7FF13150501C7
:103560003365C500678000003707000113050001BF
:10357000E364E8F4130580016FF01FF43318D800FA
:10358000B3D5E7003393D800B397D70033D7E8001B
:10359000935808013366F70033F7150393170801B2
:1035A00093D7070113550601B3D515031317070168
:1035B0003367A700B386B70213850500637ED70083
:1035C000330707011385F5FF636807016376D700AA
:1035D0001385E5FF33070701B306D74033F716031A
:1035E0001316060113560601B3D616031317070167
:1035F000B388D702B367C7001387060063FE1701BD
:10360000B38707011387F6FF63E8070163F6170125
:103610001387E6FFB387070193150501B3871741A9
:10362000B3E5E5006FF09FEB63E6D51837070100BF
:1036300063F4E6041307F00FB335D7009395350014
:103640003757008033D5B600130707B53307A700F7
:1036500003470700130500023307B700B305E54031
:103660006316E50213051000E3EEF6EE33B5C8006D
:10367000134515006FF01FEF370700019305000198
:10368000E3E0E6FC930580016FF09FFB3353E60017
:10369000B396B6003363D30013550301B31EB600CF
:1036A00033D6E700B376A602B397B70033D7E80066
:1036B0003368F7009317030193D7070113570801E5
:1036C0003356A6029396060133E7E600338FC7020E
:1036D000130E0600637EE70133076700130EF6FF43
:1036E000636867006376E701130EE6FF3307670040
:1036F0003307E741B376A7023357A7029396060133
:103700003386E7029317080193D70701B3E7F60062
:103710009306070063FEC700B38767009306F7FFB1
:1037200063E8670063F6C7009306E7FFB3876700A7
:1037300013150E01370E01003365D5009306FEFF09
:103740003378D500B387C740B3F6DE0013560501C2
:1037500093DE0E013303D802B306D60213570301DA
:103760003308D8033308D800330707013306D603DC
:103770006374D7003306C601935607013386C6002B
:1037800063E6C702E39CC7CEB70701009387F7FF44
:103790003377F700131707013373F300B398B800BA
:1037A0003307670093050000E3FEE8DA1305F5FF31
:1037B0006FF0DFCC93050000130500006FF09FDA77
:1037C0009308060013870600930705001388050079
:1037D000639C0622B7560080938606B563FCC50C31
:1037E00037030100637E660A1303F00F6374C3009E
:1037F000130780003353E600B386660003CE06004D
:10380000330EEE00130700023303C741630CC701F8
:10381000B3956500335EC501B31866003368BE001A
:10382000B317650013D608013377C8021395080152
:103830001355050193D607013358C8021317070122
:10384000B366D7003308050363FA0601B386160191
:1038500063E6160163F40601B3861601B3860641DA
:1038600033F7C6029397070193D70701B3D6C60271
:10387000B306D50213150701B367F50063FAD70045
:10388000B387170163E6170163F4D700B387170105
:10389000B387D74033D567009305000067800000E9
:1038A0003703000113070001E36666F41307800184
:1038B0006FF05FF46316060013061000B35816038A
:1038C0003706010063F2C80A1306F00F637416018D
:1038D0001307800033D6E800B386C60003CE060087
:1038E000330EEE00130700023303C7416318C70904
:1038F000B385154113D70801139508011355050128
:1039000013D60701B3F6E502B3D5E5029396060197
:10391000B3E6C600B305B50263FAB600B386160176
:1039200063E6160163F4B600B3861601B385B640AC
:10393000B3F6E5029397070193D70701B3D5E502E4
:10394000B305B50213950601B367F50063FAB70036
:10395000B387170163E6170163F4B700B387170154
:10396000B387B7406FF01FF337060001130700015C
:10397000E3E2C8F6130780016FF0DFF5B398680043
:1039800033D7C501B3176500335EC50113D50801F0
:10399000B376A702B3956500336EBE009395080118
:1039A00093D5050113560E013357A70293960601CE
:1039B000B3E6C6003387E50263FAE600B386160174
:1039C00063E6160163F4E600B38616013386E6402B
:1039D000B376A602131E0E01135E0E013356A60225
:1039E000939606013386C502B3E5C60163FAC500A6
:1039F000B385150163E6150163F4C500B3851501B0
:103A0000B385C5406FF01FEFE3EAD5E83707010043
:103A100063FCE604130EF00F3337DE001317370094
:103A2000B758008033D3E600938808B5B3886800A0
:103A300003CE0800330EEE00130700023303C74124
:103A4000631EC70363E4B600636AC500B307C540DD
:103A5000B385D5403335F5003388A540138507007D
:103A6000930508006FF09FE3B708000113070001FA
:103A7000E3E816FB130780016FF09FFA3357C60186
:103A8000B3966600336FD700B3D7C50113570F0144
:103A9000B3F8E702B39565003358C5013368B80041
:103AA00093150F0193D5050193560801331666004F
:103AB00033156500B3D7E70293980801B3E6D80041
:103AC000B38EF5029388070063FED601B386E60144
:103AD0009388F7FF63E8E60163F6D6019388E7FF72
:103AE000B386E601B386D641B3FEE6021318080199
:103AF00013580801B3D6E602939E0E01B3EE0E01F1
:103B0000B385D5029387060063FEBE00B38EEE0137
:103B10009387F6FF63E8EE0163F6BE009387E6FF46
:103B2000B38EEE01B385BE4093980801B70E010035
:103B3000B3E8F8009387FEFF33F8F80093560601C8
:103B400093D80801B377F6003307F802B387F80279
:103B50003308D802B388D8023308F8009356070117
:103B6000B386060163F4F600B388D801B7070100F5
:103B70009387F7FF13D80601B3F6F6009396060174
:103B80003377F700B30818013387E60063E61501C1
:103B9000639E1501637CE5003306C7403337C700D9
:103BA0003307E701B388E840130706003307E54011
:103BB0003335E500B3851541B385A540B397C501FD
:103BC0003357670033E5E700B3D565006FF01FCDCD
:103BD000130101F6232E1108232C8108232A9108B2
:103BE0001304010A2328210923263109232441092A
:103BF0002322510923206109232E7107232C8107D9
:103C0000232A91072328A1072326B107971700002D
:103C100093874780130101FC83A207009306F100FC
:103C2000130101FC03AF470083AE870003AEC7005A
:103C300003A3070183A8470103A8870183D5C70110
:103C400003C6E7019307F10093F707FF171700007A
:103C50001307C7D0832F070093F606FF23A857004A
:103C600093032000971200009382420623A0D20003
:103C700023A0D70023A4770097160000938646055B
:103C80009303800223A6770023A0F60023A2070057
:103C9000032547002320F4F923AAE70123ACD70129
:103CA00023AEC70123A0670223A2170323A407039F
:103CB0002396B7022387C7028347E70103238700C0
:103CC0008328C700032807018325470103268701AE
:103CD0008356C7012322A4F8171700001307070D06
:103CE000171500001305C599230FF4F89307A000DA
:103CF000232EF764232464F8232614F9232804F9D7
:103D0000232AB4F8232CC4F8231ED4F8EFE0CFCB39
:103D1000970500009385057217050000130585724D
:103D2000EFE08FCA9717000083A747F96388076AF7
:103D30001705000013054573EFE00FC937460F0064
:103D400013060624970500009385C5771705000024
:103D500013050578EFE04FC71715000013054592CE
:103D6000EFE08FC69307401F2326F4F6171A0000D2
:103D7000130ACAC09717000023A007F49719000080
:103D8000938909F4971C0000938C0CF4171D000014
:103D9000130DCD0197140000938444C00329C4F689
:103DA000170500001305057493050900EFE0CFC166
:103DB00013051000EFE01FC6F32700B0171700002F
:103DC000130747EF930D1900930A10002320F70003
:103DD00013092000EFE04FE1EFE0CFDD8347EA0178
:103DE0000357CA01832E0A00032E4A0003238A00C8
:103DF0008328CA0003280A0103264A0183268A0170
:103E0000230FF4FA930504FA93071000130504F83E
:103E1000231EE4FA232EF4F6232A24F72320D4FBCE
:103E20002322C4FB232464FA232614FB232804FB47
:103E3000232AC4FA232CD4FAEFE04FA693070500F7
:103E4000032544F793B7170017170000130787E7F8
:103E50002320F7006348A90293172500B387A70022
:103E60009387D7FF130684F793053000232CF4F6CD
:103E7000EFE00F99032544F713051500232AA4F654
:103E8000E35CA9FC832684F71306050093050D0067
:103E900013850184EFE0CF9797170000938747E3DE
:103EA00003A50700EFE0CFBA03C70900930700049A
:103EB00063F2E74E130B1004930B30006F004001C8
:103EC00083C70900130B1B00137BFB0F63E2670919
:103ED0009305300413050B00EFE00F9A8327C4F716
:103EE000E310F5FE9305C4F713050000EFE00FA201
:103EF00083C7E40103A3040083A8440003A884004B
:103F000003A5C40083A5040103A6440183A684017C
:103F100003D7C401230FF4FA83C70900130B1B0056
:103F2000232064FA232214FB232404FB2326A4FA6F
:103F30002328B4FA232AC4FA232CD4FA231EE4FA41
:103F400023A05C01137BFB0F938B0A00E3F267F95C
:103F5000032B44F7032C84F7938A1A00338B6B03EB
:103F6000130544F7B34B8B03232A74F7EFE04FA8F4
:103F7000E3925DE7F32700B017170000130747D35C
:103F800013050000130907002320F700EFE09FA8A6
:103F900017170000130707D203270700832709001C
:103FA000B387E74017170000130747D02320F70017
:103FB0006356F03E93071000171700001307C7CF92
:103FC0002320F7001705000013058557EFE0CF9F6A
:103FD000170500001305C56AEFE00F9F83A50C00CD
:103FE000170500001305455917190000130949CE9C
:103FF000EFE08F9D930550001705000013058559CC
:10400000EFE08F9C971700009387C7CB83A507002D
:10401000170500001305C559330B8B41EFE0CF9A0C
:1040200093051000170500001305C556EFE0CF9962
:104030009715000083C5D5C817050000130505595D
:10404000EFE08F9893051004170500001305C5597C
:10405000EFE08F9783C50900170500001305855A07
:1040600097140000938404C4EFE00F969305200496
:104070001705000013054557EFE00F9583A501864E
:10408000170500001305C559EFE00F949305700064
:104090001705000013050550EFE00F939717000078
:1040A0009387C7D083A5C765170500001305055979
:1040B000EFE08F91170500001305055AEFE0CF9050
:1040C000170500001305055CEFE00F90832709003A
:1040D000170500001305C55B83A50700EFE0CF8E31
:1040E000170500001305855CEFE00F8E832709009C
:1040F000170500001305C55E83A54700EFE0CF8CD0
:1041000093050000170500001305C548EFE0CF8BAD
:1041100083270900170500001305455E83A5870066
:10412000EFE08F8A930520001705000013058546F0
:10413000EFE08F8983270900170500001305C55D8F
:1041400083A5C700EFE04F88930510011705000015
:1041500013054544EFE04F8783250900170500004C
:104160001305455D17190000130949B6938505012C
:10417000EFE08F85170500001305855DEFE0CF8424
:104180001705000013054560EFE00F848327090041
:10419000170500001305C54F83A50700EFE0CF8288
:1041A000170500001305855FEFE00F8283270900E4
:1041B000170500001305C55283A54700EFE0CF8027
:1041C00093050000170500001305C53CEFD0DFFF85
:1041D00083270900170500001305455283A58700B2
:1041E000EFD09FFE93051000170500001305853AD8
:1041F000EFD09FFD83270900170500001305C55167
:1042000083A5C700EFD05FFC9305200117050000D0
:1042100013054538EFD05FFB832509001705000023
:104220001305455193850501EFD01FFA17050000CE
:1042300013050552EFD05FF9832544F717050000F9
:104240001305C559EFD05FF893055000170500001E
:1042500013054534EFD05FF793173B00338B67416D
:10426000B3057B411705000013050559EFD0DFF5B5
:104270009305D000170500001305C531EFD0DFF41A
:10428000832584F7170500001305C558EFD0DFF329
:1042900093057000170500001305C52FEFD0DFF25E
:1042A0008325C4F71705000013058558EFD0DFF10B
:1042B000170500001305052E93051000EFD0DFF061
:1042C000930504F81705000013054558EFD0DFEFFC
:1042D0001705000013054559EFD01FEF930504FAA9
:1042E000170500001305C55BEFD01FEE1705000092
:1042F0001305C55CEFD05FED1705000013054538C9
:10430000EFD09FEC8326C4F6B7470F0093870724AE
:10431000B387F60217170000130747990327070012
:10432000170500001305055DB345D702B3C7E702C3
:1043300017170000232AB79623A0F400EFE01F848C
:1043400083A50400170500001305055EEFE01F8339
:10435000130104F68320C109032481098324410940
:10436000032901098329C108032A8108832A4108F6
:10437000032B0108832BC107032C8107832C4107E2
:10438000032D0107832DC106130500001301010A47
:1043900067800000930B30006FF09FBB1705000093
:1043A00013058516EFE08FFD0327C4F617050000FF
:1043B0001305052D93172700B387E7009397170080
:1043C0002326F4F6EFE08FFB971700009387C78E44
:1043D00083A70700E384079C6FF0DFBE170500008A
:1043E0001305450BEFD05FDE6FF05F95130101FF02
:1043F000170500001305455E23261100EFE04FED81
:104400008320C1001305F0FF130101016780000044
:104410004448525953544F4E452050524F475241F1
:104420004D2C20534F4D4520535452494E470000C8
:10443000432C2056657273696F6E20322E32000055
:104440004468727973746F6E652042656E63686D3F
:1044500061726B2C2056657273696F6E2025730A2A
:104460000000000050726F6772616D20636F6D70A5
:10447000696C656420776974682027726567697361
:1044800074657227206174747269627574650A00BC
:1044900050726F6772616D20636F6D70696C6564D7
:1044A00020776974686F7574202772656769737403
:1044B000657227206174747269627574650A000000
:1044C00072646379636C6528290000005573696E16
:1044D000672025732C20485A3D25640A00000000FF
:1044E000547279696E672025642072756E7320742A
:1044F00068726F756768204468727973746F6E654F
:104500003A0A00004D656173757265642074696DC7
:104510006520746F6F20736D616C6C20746F206FF9
:10452000627461696E206D65616E696E6766756C37
:1045300020726573756C74730A00000046696E61C1
:104540006C2076616C756573206F662074686520D9
:104550007661726961626C65732075736564206948
:104560006E207468652062656E63686D61726B3A77
:104570000A000000496E745F476C6F623A20202089
:1045800020202020202020202025640A0000000078
:10459000202020202020202073686F756C6420620A
:1045A000653A20202025640A00000000426F6F6CED
:1045B0005F476C6F623A202020202020202020209E
:1045C0002025640A0000000043685F315F476C6F7C
:1045D000623A202020202020202020202025630A4D
:1045E00000000000202020202020202073686F750C
:1045F0006C642062653A20202025630A00000000D8
:1046000043685F325F476C6F623A20202020202091
:10461000202020202025630A000000004172725FE4
:10462000315F476C6F625B385D3A2020202020208C
:104630002025640A000000004172725F325F476CFF
:104640006F625B385D5B375D3A2020202025640A6D
:1046500000000000202020202020202073686F759B
:104660006C642062653A2020204E756D6265725F31
:104670004F665F52756E73202B2031300A000000A8
:104680005074725F476C6F622D3E0A002020507498
:10469000725F436F6D703A20202020202020202060
:1046A0002025640A00000000202020202020202057
:1046B00073686F756C642062653A20202028696DEC
:1046C000706C656D656E746174696F6E2D64657074
:1046D000656E64656E74290A00000000202044693C
:1046E0007363723A202020202020202020202020C8
:1046F0002025640A000000002020456E756D5F4390
:104700006F6D703A20202020202020202025640A70
:10471000000000002020496E745F436F6D703A20E6
:1047200020202020202020202025640A00000000D6
:1047300020205374725F436F6D703A202020202038
:10474000202020202025730A0000000020202020A7
:104750002020202073686F756C642062653A2020E9
:10476000204448525953544F4E452050524F4752BF
:10477000414D2C20534F4D4520535452494E470A2A
:10478000000000004E6578745F5074725F476C6F74
:10479000622D3E0A00000000202020202020202042
:1047A00073686F756C642062653A20202028696DFB
:1047B000706C656D656E746174696F6E2D64657083
:1047C000656E64656E74292C2073616D652061735C
:1047D0002061626F76650A00496E745F315F4C6FCD
:1047E000633A202020202020202020202025640A39
:1047F00000000000496E745F325F4C6F633A202006
:1048000020202020202020202025640A00000000F5
:10481000496E745F335F4C6F633A20202020202064
:10482000202020202025640A00000000456E756DC0
:104830005F4C6F633A202020202020202020202061
:104840002025640A000000005374725F315F4C6FD2
:10485000633A202020202020202020202025730AB9
:1048600000000000202020202020202073686F7589
:104870006C642062653A2020204448525953544FBA
:104880004E452050524F4752414D2C203127535412
:1048900020535452494E470A000000005374725F7F
:1048A000325F4C6F633A20202020202020202020DF
:1048B0002025730A00000000202020202020202036
:1048C00073686F756C642062653A202020444852FA
:1048D0005953544F4E452050524F4752414D2C2072
:1048E00032274E4420535452494E470A00000000DC
:1048F0004D6963726F7365636F6E647320666F7268
:10490000206F6E652072756E207468726F756768AF
:10491000204468727973746F6E653A20256C640A5E
:10492000000000004468727973746F6E65732070C4
:104930006572205365636F6E643A2020202020202A
:104940002020202020202020202020202020202067
:10495000256C640A000000004448525953544F4EDD
:10496000452050524F4752414D2C2031275354205F
:10497000535452494E4700004448525953544F4EE5
:10498000452050524F4752414D2C2032274E442053
:10499000535452494E4700004448525953544F4EC5
:1049A000452050524F4752414D2C2033275244202E
:1049B000535452494E470000286E756C6C29000014
:1049C0006D6379636C6500006D696E7374726574F4
:1049D00000000000496D706C656D656E74206D613E
:1049E000696E28292C20666F6F210A002573203DEF
:0549F0002025640A000F
:1049F80088DBFFFF24DBFFFF94DBFFFF24DBFFFFE7
:104A080024DBFFFF24DBFFFF24DBFFFFA4DBFFFF2A
:104A180024DBFFFF24DBFFFF08DBFFFFD4DDFFFF04
:104A280024DBFFFF08DBFFFF38DBFFFF38DBFFFF7E
:104A380038DBFFFF38DBFFFF38DBFFFF38DBFFFF2A
:104A480038DBFFFF38DBFFFF38DBFFFF24DBFFFF2E
:104A580024DBFFFF24DBFFFF24DBFFFF24DBFFFF5A
:104A680024DBFFFF24DBFFFF24DBFFFF24DBFFFF4A
:104A780024DBFFFF24DBFFFF24DBFFFF24DBFFFF3A
:104A880024DBFFFF24DBFFFF24DBFFFF24DBFFFF2A
:104A980024DBFFFF24DBFFFF24DBFFFF24DBFFFF1A
:104AA80024DBFFFF24DBFFFF24DBFFFF24DBFFFF0A
:104AB80024DBFFFF24DBFFFF24DBFFFF24DBFFFFFA
:104AC80024DBFFFF24DBFFFF24DBFFFF24DBFFFFEA
:104AD80024DBFFFF24DBFFFF24DBFFFF24DBFFFFDA
:104AE80024DBFFFF24DBFFFF24DBFFFF24DBFFFFCA
:104AF800ECDDFFFFD4DCFFFF24DBFFFF24DBFFFF3F
:104B080024DBFFFF24DBFFFF24DBFFFF24DBFFFFA9
:104B180024DBFFFF08DEFFFF24DBFFFF24DBFFFFB2
:104B280078DEFFFFC0DBFFFF24DBFFFF24DBFFFF96
:104B380024DDFFFF24DBFFFF84DEFFFF24DBFFFF14
:104B480024DBFFFF08DDFFFF00010202030303036C
:104B58000404040404040404050505050505050505
:104B680005050505050505050606060606060606E5
:104B780006060606060606060606060606060606CD
:104B880006060606060606060707070707070707B5
:104B9800070707070707070707070707070707079D
:104BA800070707070707070707070707070707078D
:104BB800070707070707070707070707070707077D
:104BC8000707070707070707080808080808080865
:104BD800080808080808080808080808080808084D
:104BE800080808080808080808080808080808083D
:104BF800080808080808080808080808080808082D
:104C0800080808080808080808080808080808081C
:104C1800080808080808080808080808080808080C
:104C280008080808080808080808080808080808FC
:104C380008080808080808080808080808080808EC
:084C4800080808080808080824
:104C50001000000000000000037A5200017C0101F6
:104C60001B0D02001000000018000000D0E2FFFF42
:104C70005004000000000000100000002C000000A4
:104C80000CE7FFFF340400000000000010000000EB
:104C9000400000002CEBFFFF1004000000000000AB
:040000058000000077
:00000001FF
